:020000040800F2
:10000000F0130020650100080911000849090008E3
:1000100005110008D3020008832800080000000032
:10002000000000000000000000000000C5140008EF
:1000300069060008000000007B010008C1170008E5
:100040007F0100087F0100087F0100087F01000890
:100050007F0100087F0100087F0100087F01000880
:100060007F0100087F0100087F0100087F01000870
:10007000350400087F010008390400087F010008EA
:100080007F0100087F0100087F0100087F01000850
:100090007F0100087F0100087F0100087F01000840
:1000A0007F0100087F0100087F0100087F01000830
:1000B000F1180008111900087F0100087F010008ED
:1000C0007F0100087F0100087F0100087F01000810
:1000D0007F01000809240008FD240008FF2400080F
:1000E0007F0100087F0100087F0100087F010008F0
:1000F0007F0100087F0100087F0100087F010008E0
:100100007F0100087F0100087F0100087F010008CF
:100110007F0100087F0100087F0100087F010008BF
:100120007F0100087F0100087F0100087F010008AF
:10013000DFF80CD000F09CF800480047453000087C
:10014000F0130020EFF30980704780F309887047AF
:10015000EFF30880704780F30888704740BA704713
:10016000C0BA70470648804706480047FEE7FEE7EA
:10017000FEE7FEE7FEE7FEE7FEE7FEE7FEE7FEE757
:10018000911800083101000840EA01039B0703D0E1
:1001900009E008C9121F08C0042AFAD203E011F8C6
:1001A000013B00F8013B521EF9D27047D2B201E088
:1001B00000F8012B491EFBD270470022F6E710B56C
:1001C00013460A4604461946FFF7F0FF204610BDC5
:1001D000421C10F8011B0029FBD1801A704710B592
:1001E000002200E0521C835C8C5CA34201D1002BF6
:1001F000F8D1D8B2E1B2401A10BD034611F8012B74
:1002000000F8012B002AF9D1184670472DE9F05F5C
:100210000546002092469B46884606468146402475
:100220001BE0284641464746224600F042F8534626
:100230005A46C01A914110D311461846224600F082
:1002400029F82D1A67EB01084F46224601200021AC
:1002500000F020F817EB00094E41201EA4F1010424
:10026000DFDC484631462A464346BDE8F09F0000A1
:10027000064C074D06E0E06840F0010394E80700F3
:1002800098471034AC42F6D3FFF756FF8835000884
:10029000A8350008202A04DB203A00FA02F10020E9
:1002A00070479140C2F1200320FA03F319439040B4
:1002B0007047202A04DB203A21FA02F0002170471F
:1002C00021FA02F3D040C2F12002914008431946BE
:1002D000704700BFFEE72DE9F043ADF26C4D80465C
:1002E0000E4691460DF2044000F00AFE002514E08F
:1002F000701BB0F5806F02D94FF4806700E0771B68
:10030000BAB208EB050101A802F0E6FE3A4601A9DF
:100310000DF2044000F006FE3D44B542E8D30DF274
:10032000044000F085FD002408E019F804100DF2E7
:100330005C40005D814200D002E0641C102CF4DBC4
:1003400000BF102C04DA00200DF26C4DBDE8F083E4
:100350000120F9E72DE9F047ADF5006D07460E469F
:1003600015469A462DB94FF0FF300DF5006DBDE8EA
:10037000F0877819B0F5800F02D94FF0FF30F4E71D
:10038000711906F58030814202D96FF00100ECE767
:10039000524629463846FFF79EFF10B96FF002001B
:1003A000E3E7002416E0281BB0F5806F02D94FF474
:1003B000806902E0281B1FFA80F939194A460DF5B9
:1003C000806002F089FE30194A460DF5806102F026
:1003D000DBFA4C44AC42E6D3002427E0281BB0F5FE
:1003E000806F02D94FF4806902E0281B1FFA80F960
:1003F00039194A460DF5806002F06EFE30194A4602
:10040000694600F0E1FF4FF000080CE00DF5806058
:1004100010F808001DF80810884202D06FF00300A1
:10042000A3E708F10108C845F0DB4C44AC42D5D342
:1004300000209AE77047000010B54FF4005000F01C
:10044000DFF801280AD1000300F01AF84FF4005039
:1004500000F008F80021024800F020F810BD00006C
:100460004400024010F0805F02D00349086001E0C0
:100470000249486070470000040402400000024046
:1004800010F0805F02D00349086001E00249486033
:1004900070470000040402400000024021B10268DD
:1004A00042F00102026004E002684FF6FE731A4057
:1004B0000260704701684FF6FE7211400160002132
:1004C000016041608160C1604B49884208D14A495E
:1004D0000839496841F00F01474A083A51608AE0FB
:1004E00045491431884208D143490839496841F0E7
:1004F000F001414A083A51607DE03F492831884285
:1005000008D13D490839496841F470613A4A083ACE
:10051000516070E038493C31884208D13649083989
:10052000496841F47041344A083A516063E0324905
:100530005031884208D130490839496841F4702166
:100540002D4A083A516056E02B496431884208D15F
:1005500029490839496841F47001274A083A51602D
:1005600049E025497831884208D12349083949684A
:1005700041F07061204A083A51603CE01F498842CE
:1005800006D1011F096841F00F01021F116032E01E
:100590001A491431884208D11849091F096841F0E5
:1005A000F001164A121F116025E0144928318842D3
:1005B00008D11249091F096841F470610F4A121FDE
:1005C000116018E00D493C31884208D10B49091FE0
:1005D000096841F47041094A121F11600BE0074994
:1005E0005031884207D10549091F096841F470213B
:1005F000024A121F116070470800024008040240BE
:1006000001460020002211F0805F02D0054B1A68DD
:1006100001E0054B1A680A4201D0012000E00020E9
:1006200070470000000402400000024010B50022A4
:10063000026847F6F0739A430C6A8B6823430C698F
:1006400023434C6923438C692343CC6923434C6A7D
:1006500023438C6A23431A430260CB6843600B68D0
:1006600083604B68C36010BD704710B5024606E05A
:10067000002102E000BF4B1CD9B22D29FADB130088
:10068000A2F10104A2B2F3D110BD000008B501210E
:10069000042000F0CDFD4FF40060ADF80000102004
:1006A0008DF8030003208DF802006946014800F030
:1006B0008CF808BD0008014030B5044604254FF40D
:1006C000302000F06FF80546042D17D10C48006962
:1006D00040F002000A49086108464461006940F0A0
:1006E000400008614FF4302000F05CF805460448F3
:1006F000006941F6FD71084001490861284630BD96
:100700000020024004200B49C96811F0010F01D0FC
:1007100001200EE00749C96811F0040F01D0022042
:1007200007E00449C96811F0100F01D0032000E070
:1007300004207047002002400348006940F0800018
:1007400001490861704700000020024070B504466E
:100750000D460426F00200F025F80646042E11D1BD
:100760000948006940F00100074908612580F0024E
:1007700000F018F806460448006941F6FE7108408A
:1007800001490861304670BD00200240024803491B
:1007900048600348486070472301674500200240D5
:1007A000AB89EFCD00B502460423FFF7ABFF03464C
:1007B00003E0FFF7A7FF0346521E012B01D1002AD9
:1007C000F7D102B90523184600BD2DE9F0410246D4
:1007D00000250026002000230024002791F803C0F4
:1007E0000CF00F0591F803C01CF0100F03D091F826
:1007F00002C04CEA050591F800C0BCF1000F31D0F1
:10080000146800202BE04FF0010C0CFA00F3B1F853
:1008100000C00CEA03069E4220D183004FF00F0C6B
:100820000CFA03F7BC4305FA03FC4CEA040491F804
:1008300003C0BCF1280F06D14FF0010C0CFA00FCEC
:10084000C2F814C00AE091F803C0BCF1480F05D10A
:100850004FF0010C0CFA00FCC2F810C0401C082834
:10086000D1D31460B1F800C0BCF1FF0F34DD54687F
:1008700000202EE000F1080C4FF0010808FA0CF3FC
:10088000B1F800C00CEA03069E4221D183004FF06C
:100890000F0C0CFA03F7BC4305FA03FC4CEA040402
:1008A00091F803C0BCF1280F05D100F1080C08FA3B
:1008B0000CF8C2F8148091F803C0BCF1480F07D1BE
:1008C00000F1080C4FF0010808FA0CF8C2F810808B
:1008D000401C0828CED35460BDE8F08102460020B9
:1008E000D3680B4201D0012000E000207047416135
:1008F0007047016170470AB1016100E041617047D2
:100900003EB55824684600F00FF8002503E01DF8B6
:10091000050044406D1C0C2DF9DB04B95824FF2C54
:1009200000D1852420463EBD0021064A00BF05E0D7
:1009300013780370401C521C4B1CD9B20C29F7DBF6
:1009400070470000E8F7FF1F0948C08808498988F8
:100950000843074949880843054909880843054968
:1009600008800846018804A002F040F800BFFEE7B6
:1009700004000020140000200D0A5B4846483D2575
:100980003034785D0D0A000010B51148406A40F01F
:1009900001000F49486200BF0D48406AC0F34000A3
:1009A0000028F9D07D2000F0E7FC08B100F050FCF1
:1009B00045F2555000F02AF8062000F01BF84FF4DD
:1009C000FA7000F01DF800F00DF800F003F810BD0B
:1009D000001002404CF6CC4001490860704700000E
:1009E000003000404AF6AA20014908607047000024
:1009F000003000400149486070470000003000406E
:100A000001498860704700000030004001490860DB
:100A100070470000003000402DE9F043ADF26C4D0E
:100A2000074688464FF000090DF2044000F068FACE
:100A30000025002417E01E49601800F031FD06462D
:100A400028466D1C01A90E54320A28466D1C0A5412
:100A5000B5F5806F06D14FF480620DF2044000F0CE
:100A600061FA0025A41CBC42E5D32DB12A4601A998
:100A70000DF2044000F056FA0DF2044000F0D8F9EF
:100A8000002408E018F804100DF25C40005D81427B
:100A900000D002E0641C102CF4DB00BF102C04DA40
:100AA00000200DF26C4DBDE8F0830120F9E7000055
:100AB0000040000870B504460D46074884420AD13C
:100AC0004FF480622946054800F0BCFA06463146DC
:100AD000024801F0B3FE70BD504354416500002050
:100AE00070B504460548844207D1054800F0DCFA99
:100AF00005462946024801F0A1FE70BD504354410D
:100B0000650000202DE9F04FA1B0804644462068E2
:100B10007A49884208D020687949884204D04FF049
:100B2000FF3021B0BDE8F08F2079802802D06FF02F
:100B30000100F6E773A11DA801F068FFA11D1DA823
:100B4000FFF74DFB10B16FF00200EAE794F805A043
:100B5000208B0190BAF1000F25D10198142802D002
:100B60006FF00300DDE7C34610220BF11A0166485F
:100B7000FFF70AFBD846DBF82A00644908600846FC
:100B8000006810B96FF00400CBE7002060490860EE
:100B9000604908606049086020685D490968FFF79E
:100BA00089FF0120BDE7BAF1020F7DD1474600263B
:100BB00008E05548815D07F11A00805D814200D050
:100BC00002E0761C102EF4DB00BF102E08DA53A0D2
:100BD00000F0DEF82068FFF783FF6FF00500A0E764
:100BE000D7F82E50D7F82A000290022D0CD348498E
:100BF00002980968884207D1454800682918434887
:100C00000068801C814208D949A000F0C1F8206822
:100C1000FFF766FF6FF0060083E7AD1E2A4607F177
:100C20003201002002F04AF9814607F13200691CC6
:100C3000405C00021C9007F13200405D1C990844A2
:100C400080B21C901C9949450AD041A000F0A0F840
:100C500020682F490968FFF72DFF6FF0070060E754
:100C60002068274988420DD1002609E007F13200AB
:100C7000805D3D490978484007F132018855761C6E
:100C8000AE42F3D307F1320229462148006800F052
:100C9000B9F82148006828441F4908601C480068CA
:100CA00028441B49086000E026E01B4800681749FB
:100CB0000968884210DB144914480068FFF7ACFE4D
:100CC00040B92AA000F064F82068FFF709FF6FF030
:100CD000080026E7002024E70D482AA1026803A89F
:100CE00001F094FE03A800F053F820680849096851
:100CF000FFF7E0FE022014E700BF12E7464F544121
:100D00005043544130000000A40400203C00002067
:100D10004400002048000020400000204D443520C1
:100D20004D6F64696679215265444F210D0A0000B8
:100D30004C656E677468206F72204F6666736574C9
:100D4000206572726F72215265444F210D0A0000B6
:100D5000436865636B20435243206572726F722152
:100D60005265444F210D0A00160000204368656358
:100D70006B204D4435206572726F72215265444F6D
:100D8000210D0A004C4F41443D25640D0A0000002E
:100D90007CB5054617A103C9CDE900016C464FF4A7
:100DA0008070164908600BE02178154801F0A5FC19
:100DB00000BF4021124801F0D3FB0028F9D0641C89
:100DC00020780028F0D12C460BE021780C4801F067
:100DD00094FC00BF40210A4801F0C2FB0028F9D072
:100DE000641C20780028F0D14FF480700349091D5D
:100DF00008607CBD5B4D53475D000000100801405A
:100E0000003801402DE9F04104460D461646002702
:100E100014F0010F02D00020BDE8F081AAB203490E
:100E20006018314601F0B0FD0120F5E700400008F0
:100E30002DE9F04190B0044620680E9060680F9054
:100E40002088C0F3C507382F02DAC7F1380001E067
:100E5000C7F17800804642462849204600F062F8F3
:100E60000026002518E004F11800E91C405C020689
:100E700004F11800A91C405C42EA004204F1180089
:100E8000691C405C42EA002004F11801495D0843F6
:100E90004DF82600761C2D1D0E2EE4D3694604F174
:100EA000080000F03FFE0026002521E004F10800C4
:100EB00010F8261050304155503830F82600C0F355
:100EC000072204F15800691C4254503850F826009B
:100ED000C0F3074204F15800A91C4254503850F89E
:100EE0002600000E04F15801EA1C8854761C2D1DC2
:100EF000042EDBD310B0BDE8F081000048350008B7
:100F000000214160016005498160054AC260CA4311
:100F10000261034AD24342617047000001234567E2
:100F200089ABCDEF2DE9F04391B004460F4615464D
:100F30002088C0F3C509206800EBC50021688842FD
:100F400002D26068401C6060206800EBC500206031
:100F5000606800EB5570606033E017F8012B48467D
:100F600009F1010904F118010A54B9F1400F28D11F
:100F70004FF0000800261AE004F11800F11C405C54
:100F8000020604F11800B11C405C42EA004204F180
:100F90001800711C405C42EA002004F11801895DD0
:100FA000084301A941F8280008F10108361DB8F1ED
:100FB000100FE1D301A904F1080000F0B3FD4FF0D8
:100FC00000092800A5F10105C7D111B0BDE8F083E3
:100FD00008B54FF4A06000F0D3F825208DF800008C
:100FE00001208DF801008DF802008DF8030068469D
:100FF00000F08CF827208DF8000001208DF801000A
:101000008DF802008DF80300684600F07FF80E208E
:101010008DF8000001208DF801008DF802008DF898
:101020000300684600F072F80C208DF800000120E3
:101030008DF801008DF802008DF80300684600F07D
:1010400065F808BD2DE9F04104460E4617462546D1
:1010500032212846FFF7B1F80F4828608020287118
:10106000022068710DA1A81D01F0D0FC0C48008879
:10107000401C80B20A490880E88218202883102288
:10108000084905F11A00FFF77FF8C5F82A60C5F88E
:101090002E703220BDE8F0815043544130000000F2
:1010A00038000020A404002070B5044625462C21F9
:1010B0002846FFF782F80D4828608020287100201C
:1010C00068710BA1A81D01F0A1FC0A480078E88214
:1010D0001220288308A105F11A00FFF78EF80020DE
:1010E0006885074908802C2070BD0000504354419A
:1010F00030000000160000204E554C4C000000004F
:101100003800002000BFFEE77047000070B50021E6
:1011100000230F22C4780CB3164C246804F4E06456
:10112000C4F5E064210AC1F10403CA40447804FA1A
:1011300003F184781440214309010F4C0678A1552E
:10114000047804F01F050124AC4005786D114FF0C0
:10115000E02606EB8505C5F8004109E0047804F0B7
:101160001F050124AC40054D0678761145F8264050
:1011700070BD00000CED00E000E400E080E100E064
:1011800002490143024A1160704700000000FA055D
:101190000CED00E004490978044A11700249087016
:1011A0000121034A117170473500002036000020EC
:1011B000300000200021C1800160704701460868AE
:1011C000A8B1C28812B1C288521EC280C28872B948
:1011D0000022828007E0006820B1C28812B9002294
:1011E000828000E001E00028F5D100BF0860704770
:1011F00029B1064A52690243044B5A6104E0034A8A
:1012000052698243014B5A6170470000001002404E
:1012100029B1064AD2690243044BDA6104E0034A69
:10122000D2698243014BDA6170470000001002402E
:1012300029B1064A92690243044B9A6104E0034AC9
:1012400092698243014B9A6170470000001002408E
:101250000348406A40F080700149486270470000CE
:101260000010024010B501211C20FFF7C1FF012131
:101270004802FFF7DDFF01210846FFF7B9FF012112
:101280008803FFF7D5FF01210846FFF7C1FF0020C3
:101290000149086010BD00000000002030B50021A9
:1012A0000022002400232D4D6D6805F00C0121B1B2
:1012B000042905D0082923D105E0294D056022E045
:1012C000284D05601FE0254D6D6805F47012234D13
:1012D0006D6805F48034022505EB92421CB9224D5D
:1012E000554305600BE01D4D6D6815F4003F03D0BC
:1012F0001E4D5543056002E01A4D5543056002E05E
:10130000174D056000BF00BF144D6D6805F0F0017A
:101310000909174D6B5C0568DD4045600F4D6D6830
:1013200005F4E061090A124D6B5C4568DD4085609B
:101330000A4D6D6805F46051C90A0D4D6B5C456836
:10134000DD40C560054D6D6805F44041890B094DD0
:101350006B5CC568B5FBF3F5056130BD001002405C
:1013600000127A00001BB70000093D00808D5B0071
:101370007C0000208C00002010B5014600220023D4
:1013800000204A11012A02D1094C236806E0022AF2
:1013900002D1074C236A01E0054C636A01F01F0289
:1013A000012494401C4201D0012000E0002010BD27
:1013B0000010024010B520220021024801F08CFEEE
:1013C00010BD0000CE040020F0B505460B461646C1
:1013D000002700240DE0281900F062F80246384684
:1013E0007F1C1A544FEA122C38467F1C03F800C0A9
:1013F000A41CB442EFDBF0BD21B1028842F04002F0
:10140000028004E002884FF6BF731A4002807047E2
:101410000246002013890B4201D0012000E0002089
:1014200070470146888970478181704710B5002256
:10143000028802F441520B884C8823438C88234352
:10144000CC8823430C8923434C8923438C89234331
:10145000CC8923431A430280838B4FF2FF742340CD
:1014600083830B8A038210BD10B5044600BF02219E
:101470000A48FFF7CDFF0028F9D021460748FFF7BB
:10148000D3FF00BF01210548FFF7C2FF0028F9D0B4
:101490000248FFF7C6FFC0B210BD00000030014097
:1014A000014608887047000010B50548FFF782FE26
:1014B0004FF47A7000F0F2FA00F020FB10BD00004B
:1014C000740000207047000010B52022002102485F
:1014D00001F076FE10BD0000CE04002010B500F033
:1014E00001F810BD0CB50020019000903048006854
:1014F00040F480302E49086000BF2D48006800F499
:10150000003000900198401C0190009818B9019893
:10151000B0F5A06FF1D12648006810F4003F02D06A
:101520000120009001E000200090009801283ED1A9
:101530002048006840F010001E4908600846006816
:1015400020F00300086008460068086018484068FA
:101550001749486008464068486008464068486047
:101560000846406820F47C1048600846406840F413
:10157000302048600846006840F08070086000BF76
:101580000B48006810F0007FFAD00948406820F04E
:101590000300074948600846406840F00200486080
:1015A00000BF0348406800F00C000828F9D10CBDCA
:1015B000001002400020024030B502460B4619469A
:1015C000144607E008782578A84201D0012030BDF4
:1015D000491C641C08780028F4D100BFF7E700001C
:1015E00070B506460C460748007800B170BD20462D
:1015F000FEF7EEFD05462946204601F01FF900BF23
:10160000F4E700006000002010B5002400202B4902
:1016100008602B4908602B480078122804D0342831
:1016200003D0782847D107E045E027A0FFF7B0FBBB
:101630002848FFF755FA3EE027480079462837D179
:10164000254840796F2833D12348807954282FD1F9
:101650002148C07961282BD11F49CA69886901F1E5
:1016600008031E49FEF776FE98B11DA0FFF790FB18
:101670001949CA69886901F108031849FEF76AFE29
:1016800018B11DA0FFF784FB06E020A0FFF780FB48
:1016900002E022A0FFF77CFB46200F49087154218D
:1016A0000D4841714F2181714B21C171FFF70CFF32
:1016B00001F034FC00BF00BF10BD0000200000207E
:1016C0001C000020350000205374617274444C21CA
:1016D0000D0A000050435441CE0400200040000891
:1016E000436F707920417070204661696C2172658A
:1016F000646F2E2E2E0D0A00436F7079204170709A
:10170000204661696C210D0A00000000436F70796A
:1017100020417070204F4B21310D0A00436F7079CA
:1017200020417070204F4B21320D0A0070B5FFF739
:1017300099FD00F06DFEFFF74BFC1C480068642229
:10174000B0FBF2F1B1F1807F00D31DE021F07F40CA
:10175000401E4FF0E022506150170F22002807DA98
:1017600013071D0E124B00F00F04241F1D5503E03C
:1017700013071C0E0F4B1C5400BF00204FF0E0223B
:1017800090610720106100BFFEF780FF01F07CF838
:10179000FFF7B6F808490870084800210160017198
:1017A000FFF782FE1220FFF7F5FC70BD90000020CD
:1017B00018ED00E000E400E01600002030000020FA
:1017C00010B501201D4988701D480068401C1C4947
:1017D0000860322815DB4FF400611A48FFF77EF8E5
:1017E00008B9012000E00020044622464FF40061C1
:1017F0001448FFF780F800201149086001200F49C4
:10180000C87011480078012817D110480068401CA2
:101810000E49086008460068B0F5FA7F0DDD0C48F7
:101820000CA109684160FFF74FFE0CA10020FFF7F3
:10183000D7FEFFF7A9F800BFFEE710BD300000207B
:101840000C000020000801401800002010000020BB
:10185000CE04002046544F4B00000000777269749C
:1018600065204578466C617368206572726F7221DD
:101870000D0A7265626F6F74204D435520616E646E
:1018800020476F746F20415050210D0A0000000066
:1018900010B51348006840F001001149086008467F
:1018A0004068104908400E494860084600680E49E3
:1018B00008400B4908600846006820F48020086052
:1018C0000846406820F4FE0048604FF41F0088601E
:1018D000FFF704FE4FF000600449086010BD0000EF
:1018E000001002400000FFF8FFFFF6FE08ED00E0E8
:1018F00010B50121880700F02BF830B10348FFF73D
:101900005DFC0121880700F014F810BD7400002070
:1019100010B50121044800F01BF818B1012102485C
:1019200000F007F810BD000000040040CA43028226
:101930007047CA430282704721B1028842F0010217
:10194000028004E002884FF6FE731A40028070475E
:1019500030B50246002000230024158A05EA010361
:10196000958905EA010413B10CB1012000E00020C3
:1019700030BD1AB183890B43838102E083898B4395
:101980008381704781847047002202881D4B9842F2
:101990000ED01D4B98420BD0B0F1804F08D01B4B9E
:1019A000984205D01A4B984202D01A4B984204D163
:1019B0004FF68F731A404B881A43174B984207D043
:1019C000164B984204D04FF6FF431A40CB881A4377
:1019D00002808B8883850B8803850A4B98420BD045
:1019E000094B984208D00E4B984205D00D4B9842B7
:1019F00002D00D4B984201D10B7A038601238382DA
:101A000070470000002C01400034014000040040F9
:101A100000080040000C004000100040001400408E
:101A200000400140004401400048014010B5164804
:101A30000068401C04D014480068401C124908602B
:101A400012480078122804D034280AD0782817D1F8
:101A500008E00D480068042802D97820FFF79AFBB7
:101A60000EE00DE008480068042800D210BD0648CA
:101A7000007810F0010F02D005A0FFF789F900BF30
:101A800000BF00BFF2E7000020000020350000206A
:101A90004E4F20415050210D0A0000001FB5044652
:101AA00001210846FFF7B4FBADF808401148006873
:101AB0001149B0FBF1F0401E80B2ADF804000020E7
:101AC000ADF80A00ADF8060001A94FF08040FFF71D
:101AD0005BFF1C208DF8000001208DF801008DF8BF
:101AE00003006846FFF712FB01218807FFF71EFF7E
:101AF0001FBD00009000002040420F0010B50121E2
:101B00008807FFF713FF00214FF08040FFF73AFFEF
:101B1000012241218807FFF72CFF01218807FFF7E9
:101B20000BFF10BDF0B505460C4628686968AA6829
:101B3000EB6801EA020623EA01073E4327683E44B8
:101B4000FE4F3E443044C60146EA5060084400EA75
:101B5000010622EA00073E4367683E44F84F3E44D0
:101B600033441E0346EA1353034403EA000621EA02
:101B700003073E43A7683E44F24F3E4432445604B6
:101B800046EAD2321A4402EA030620EA02073E433A
:101B9000E7683E44EC4F3E4431448E0546EA9121CD
:101BA000114401EA020623EA01073E4327693E4445
:101BB000E64F3E443044C60146EA5060084400EA1D
:101BC000010622EA00073E4367693E44E04F3E4477
:101BD00033441E0346EA1353034403EA000621EA92
:101BE00003073E43A7693E44DA4F3E44324456045D
:101BF00046EAD2321A4402EA030620EA02073E43CA
:101C0000E7693E44D44F3E4431448E0546EA912173
:101C1000114401EA020623EA01073E43276A3E44D3
:101C2000CE4F3E443044C60146EA5060084400EAC4
:101C3000010622EA00073E43676A3E44C84F3E441D
:101C400033441E0346EA1353034403EA000621EA21
:101C500003073E43A76A3E44A6F524464F3E32445E
:101C6000560446EAD2321A4402EA030620EA020780
:101C70003E43E76A3E44BB4F3E4431448E0546EA4C
:101C80009121114401EA020623EA01073E43276B32
:101C90003E44B54F3E443044C60146EA50600844D5
:101CA00000EA010622EA00073E43676B3E44AF4F5D
:101CB0003E4433441E0346EA1353034403EA00063A
:101CC00021EA03073E43A76B3E44A94F3E443244FA
:101CD000560446EAD2321A4402EA030620EA020710
:101CE0003E43E76B3E44A34F3E4431448E0546EAF3
:101CF0009121114401EA030622EA03073E43676883
:101D00003E449D4F3E443044460146EAD06008447C
:101D100000EA020621EA02073E43A7693E44974FC4
:101D20003E4433445E0246EAD353034403EA0106C9
:101D300020EA01073E43E76A3E44914F3E44324465
:101D4000960346EA92421A4402EA000623EA000792
:101D50003E4327683E448B4F3E4431440E0546EADD
:101D60001131114401EA030622EA03073E43676981
:101D70003E44854F3E443044460146EAD060084424
:101D800000EA020621EA02073E43A76A3E447F4F6B
:101D90003E4433445E0246EAD353034403EA010659
:101DA00020EA01073E43E76B3E44794F3E4432440C
:101DB000960346EA92421A4402EA000623EA000722
:101DC0003E4327693E44734F3E4431440E0546EA84
:101DD0001131114401EA030622EA03073E43676A10
:101DE0003E446D4F3E443044460146EAD0600844CC
:101DF00000EA020621EA02073E43A76B3E44674F12
:101E00003E4433445E0246EAD353034403EA0106E8
:101E100020EA01073E43E7683E44614F3E443244B6
:101E2000960346EA92421A4402EA000623EA0007B1
:101E30003E43276A3E445B4F3E4431440E0546EA2A
:101E40001131114401EA030622EA03073E43676B9E
:101E50003E44554F3E443044460146EAD060084473
:101E600000EA020621EA02073E43A7683E444F4FBC
:101E70003E4433445E0246EAD353034403EA010678
:101E800020EA01073E43E7693E44494F3E4432445D
:101E9000960346EA92421A4402EA000623EA000741
:101EA0003E43276B3E44434F3E4431440E0546EAD1
:101EB0001131114481EA02065E4067693E443E4F9B
:101EC0003E443044060146EA1070084480EA0106A8
:101ED0005640276A3E44394F3E443344DE0246EAC8
:101EE0005353034483EA00064E40E76A3E44344FAE
:101EF0003E443244160446EA12421A4482EA030679
:101F00004640A76B3E442F4F3E443144CE0546EA3F
:101F10005121114481EA02065E4067683E442A4F1F
:101F20003E443044060146EA1070084480EA010647
:101F3000564027693E44254F3E4449E078A46AD77D
:101F400056B7C7E8DB702024EECEBDC1AF0F7CF5DD
:101F50002AC68747134630A8019546FDD898806960
:101F6000AFF7448BBED75C892211906B937198FDBB
:101F70008E4379A62108B44962251EF640B340C0BD
:101F8000515A5E26AAC7B6E95D102FD653144402F3
:101F900081E6A1D8C8FBD3E7E6CDE121D60737C358
:101FA000870DD5F4ED145A4505E9E3A9F8A3EFFC34
:101FB000D9026F678A4C2A8D4239FAFF81F6718700
:101FC00022619D6D0C38E5FD44EABEA4A9CFDE4B2D
:101FD0003344DE0246EA5353034483EA00064E408C
:101FE000E7693E449F4F3E443244160446EA12429B
:101FF0001A4482EA03064640A76A3E449A4F3E448A
:102000003144CE0546EA5121114481EA02065E4080
:10201000676B3E44954F3E443044060146EA1070DB
:10202000084480EA0106564027683E44904F3E44EB
:102030003344DE0246EA5353034483EA00064E402B
:10204000E7683E448B4F3E443244160446EA12424F
:102050001A4482EA03064640A7693E44864F3E443E
:102060003144CE0546EA5121114481EA02065E4020
:10207000676A3E44814F3E443044060146EA107090
:10208000084480EA01065640276B3E447C4F3E449C
:102090003344DE0246EA5353034483EA00064E40CB
:1020A000E76B3E44774F3E443244160446EA124200
:1020B0001A4482EA03064640A7683E44724F3E44F3
:1020C0003144CE0546EA5121114461EA03065640E7
:1020D00027683E446D4F3E443044860146EA906096
:1020E000084460EA02064E40E7693E44684F3E44B9
:1020F00033449E0246EA9353034463EA0106464092
:10210000A76B3E44634F3E443244D60346EA5242F4
:102110001A4462EA00065E4067693E445E4F3E44F0
:1021200031444E0546EAD121114461EA0306564086
:10213000276B3E44594F3E443044860146EA906046
:10214000084460EA02064E40E7683E44544F3E446D
:1021500033449E0246EA9353034463EA0106464031
:10216000A76A3E444F4F3E443244D60346EA5242A9
:102170001A4462EA00065E4067683E444A4F3E44A5
:1021800031444E0546EAD121114461EA0306564026
:10219000276A3E44454F3E443044860146EA9060FB
:1021A000084460EA02064E40E76B3E44404F3E441E
:1021B00033449E0246EA9353034463EA01064640D1
:1021C000A7693E443B4F3E443244D60346EA52425E
:1021D0001A4462EA00065E40676B3E44364F3E4456
:1021E00031444E0546EAD121114461EA03065640C6
:1021F00027693E44314F3E443044860146EA9060B0
:10220000084460EA02064E40E76A3E442C4F3E44D2
:1022100033449E0246EA9353034463EA0106464070
:10222000A7683E44274F3E443244D60346EA524212
:102230001A4462EA00065E40676A3E44224F3E440A
:1022400031444E0546EAD12111442E6806442E60E1
:102250006E680E446E60AE681644AE60EE681E4452
:10226000EE60F0BD604BBBF670BCBFBEC67E9B2867
:10227000FA27A1EA8530EFD4051D880439D0D4D9D6
:10228000E599DBE6F87CA21F6556ACC4442229F42C
:1022900097FF2A43A72394AB39A093FCC3595B65EE
:1022A00092CC0C8F7DF4EFFFD15D84854F7EA86FBB
:1022B000E0E62CFE144301A3A111084E827E53F7E1
:1022C00035F23ABDBBD2D72A91D386EB08B540F29E
:1022D0002441174800F051F940B315480088009098
:1022E0001348001D008800901248C06D40F2524112
:1022F000081A009000210F485830FEF7CFF80E481A
:10230000007850B90D490E48009AFDF73DFF0D4980
:102310000098088001200849087040F252400549A1
:10232000C865012103485830FEF7B8F808BD000021
:102330000038014000000240300000204009002029
:10234000EE0400204C00002008B540F2255127483B
:1023500000F013F9002839D0244800F0C9F9C0B2C0
:1023600000902348007801280AD19DF800102148E8
:1023700000F0C3F940F225511C4800F0CDF808BD2B
:102380001D480088B0F5167F15DA9DF800001B493E
:102390001B4A128888541A480088401C80B2184989
:1023A0000880B0F5167F01DB002008801248008805
:1023B000401C1149088000F063FA40F225510B4897
:1023C00000F0AAF89DF800000E490870082107489F
:1023D00000F0C6F8012806D1044800F089F9082168
:1023E000024800F090F800BFC9E700000048004034
:1023F00060000020003801405A000020920D0020AB
:10240000580000206400002010B5FFF75FFF10BDEA
:1024100000B585B0012144F20400FEF709FF4FF436
:102420000070ADF8100018208DF8130003208DF80F
:10243000120004A92F48FEF7C8F94FF48060ADF8E8
:10244000100004208DF8130003208DF8120004A959
:102450002848FEF7BAF94FF48070ADF8100010204C
:102460008DF8130003208DF8120004A92148FEF70F
:10247000ACF94FF4E13000900020ADF80400ADF865
:102480000600ADF80800ADF80C000C20ADF80A000D
:102490006946194800F0C0F80121174800F04BF8D0
:1024A0004021154800F02FF8002240F22771124811
:1024B00000F08DF8002240F225510F4800F087F817
:1024C000012240F224410C4800F081F80122402111
:1024D000094800F03CF801228021074800F037F855
:1024E00000F010F94FF4807002491431086005B013
:1024F00000BD00000008014000380140704710B5E1
:10250000FFF722FF10BD01F40072B2F5007F00D189
:1025100000BFCA430280704710B500220023A1F516
:1025200010646A3C00D100BF0A1201249440A3B297
:10253000DC43048010BD21B1828942F400528281C3
:1025400004E082894DF6FF731A40828170471AB108
:10255000838A0B43838202E0838A8B4383827047A2
:1025600002460020B1F5007F00D100BF13880B4266
:1025700001D0012000E00020704770B50246002421
:10258000002300250020A1F510666A3E00D100BF9F
:10259000C1F3421501F01F03012606FA03F3012DD2
:1025A00002D19689334006E0022D02D1168A3340CB
:1025B00001E0968A33400C12012606FA04F41688CC
:1025C000344013B10CB1012000E0002070BDF0B523
:1025D00003460024002600250020A1F510676A3F6D
:1025E00000D100BF1846C1F3421401F01F060127B5
:1025F00007FA06F5012C01D10C3004E0022C01D1C0
:10260000103000E014301AB107682F43076002E071
:102610000768AF430760F0BD2DE9F04786B0054677
:102620000E460024A24600BFA1460027B08900B193
:1026300000BF2F462C8A4CF6FF700440F0880443FC
:102640002C82AC894EF6F3100440B08831890843DF
:10265000718908430443AC81AC8A4FF6FF400440C3
:10266000B0890443AC8201A8FEF718FE1F488742D8
:1026700002D1DDF810A001E0DDF80CA0A88910F46B
:10268000004F08D00AEBCA0000EB0A10316849007D
:10269000B0FBF1F807E00AEBCA0000EB0A10316862
:1026A0008900B0FBF1F86420B8FBF0F004012009C8
:1026B000642101FB1089A88910F4004F08D0322052
:1026C00000EBC900B0FBF1F000F00700044308E0A4
:1026D000322000EB09106421B0FBF1F000F00F0094
:1026E00004432C8106B0BDE8F087000000380140AB
:1026F00001468888C0F308007047C1F30802828051
:102700007047000000B58BB001210846FEF770FD50
:102710001148FDF7CFFE11480090114801900020AC
:10272000029040F2524003900020049080200590D7
:1027300000200690079008904FF400500990002068
:102740000A9069460448FDF771FF01210248FDF730
:10275000A5FE0BB000BD0000580002400438014047
:102760004009002010B52548007812280ED124A178
:102770002748FEF721FF28B9FEF706F93420FEF7B7
:1027800009FD02E023A0FEF703FB10BD1B48007803
:10279000342800D0F9E71E48007850280BD11C4897
:1027A0004078432807D11A488078542803D1184824
:1027B000C078412800D0E8E71548007980281BD16F
:1027C000FEF710F9154801881148FEF79BF90446F9
:1027D00034B913A0FEF7DCFA7820FEF7DBFCD4E76F
:1027E00014F1020F08DA14F1060F05DD10A0FEF750
:1027F000CFFA7820FEF7CEFC00BFC6E735000020F8
:10280000444F574E4C4F41445F4150500000000030
:10281000EE0400202D2D2D2D0D0A00004C0000206F
:10282000436F6D706C65746564210D0A00000000D3
:102830004941502053746F70210D0A0070B5054650
:102840000E464FF480700C49086000240BE0295DAF
:102850000A48FFF752FF00BF40210848FFF780FEFB
:102860000028F9D0641CB442F1DB4FF480700249B7
:10287000091D086070BD00001008014000380140CB
:10288000704700BFFEE7000010B586B000F038F8D2
:1028900010211948FEF72DF80020ADF804004FF480
:1028A0008270ADF806000020ADF808000220ADF8F7
:1028B0000A000120ADF80C004002ADF80E0008201F
:1028C000ADF810000020ADF812000720ADF814009C
:1028D00001A90A48FEF7AAFD01210848FEF78CFD70
:1028E0004FF47A70FDF7C1FE00F0CEFC00F022FC40
:1028F0000446012006B010BD000801400030014030
:1029000008B501210420FEF793FC01210803FEF71E
:102910008FFC2020ADF8000003208DF80200182065
:102920008DF8030069461648FDF74FFF8020ADF88B
:10293000000069461248FDF748FF4020ADF800004E
:1029400004208DF8030069460D48FDF73EFF102076
:10295000ADF800008DF8030069460948FDF735FF22
:102960000120ADF8000010208DF8030069460548ED
:10297000FDF72BFF01210348FDF7B9FF08BD00005B
:1029800000080140000C01402DE9F04705460E46C5
:102990009046B5F1006F02D31348854202D3A24698
:1029A000BDE8F087A805800D00D0F9E7FDF7EEFE41
:1029B0002846FDF781FE0746042F00D0F0E70024EB
:1029C0000CE0315D601C305C01EB00201FFA80F9E7
:1029D00028194946FDF7BAFEA01C84B24445F0DB35
:1029E000FDF7AAFE00BFDBE7000001080FB4054BAE
:1029F00010B503A9044A029800F02CF810BC5DF849
:102A000014FB0000F92E0008680000200FB4084BEA
:102A100010B504A902AA039800F01CF8044602A904
:102A2000002000F046FA204610BC5DF814FB0000C0
:102A3000B32E000802E008C8121F08C1002AFAD10C
:102A400070477047002001E001C1121F002AFBD12E
:102A5000704700002DE9FF4F8DB00F460546002658
:102A6000DEE1252874D100246D1CF149A246A1465F
:102A700001222B78203B02FA03F0084202D00443E3
:102A80006D1CF6E728782A2810D06FF02F022878DE
:102A9000A0F13001092915D80AEB8A0102EB4101A6
:102AA00044F0020400EB010A6D1CF0E757F804AB98
:102AB000BAF1000F03DA44F40054CAF1000A44F0FA
:102AC00002046D1C28782E2817D115F8010F44F048
:102AD00004042A280ED06FF02F022878A0F13001CC
:102AE00009290AD809EB890102EB410100EB010930
:102AF0006D1CF2E757F8049B6D1C28786C280FD0EA
:102B000006DC4C2817D068280DD06A2814D104E0C0
:102B1000742810D07A280FD10DE044F400140AE094
:102B200044F4801401E044F440146978814202D1F5
:102B30006D1C04F580146D1C2A786E2A20D00DDCE3
:102B4000632A33D005DC002A6FD0582A12D1A2E0C4
:102B500011E0642A6AD0692A0CD167E0732A2FD069
:102B600004DC6F2A6FD0702A04D199E0752A6BD0EB
:102B7000782A6AD01046DDE90F129047761C4EE1A4
:102B8000C4F30250022806D003280AD0042801CF3B
:102B90000AD0066043E101CF4FEAE671C0E9006167
:102BA0003DE101CF06803AE1067038E117F8040BE9
:102BB0008DF8000000208DF80100EB46012003E0B5
:102BC00057F804BB4FF0FF3061074FF0000102D40B
:102BD0000DE008F10101884649450FDA8045F8DB30
:102BE0001BF808100029F4D108E008F1010188461B
:102BF0008142FADB1BF808100029F6D1DDE90F232A
:102C0000AAEB08008146214600F03BF9304400EB76
:102C1000080604E0DDE90F121BF8010B9047B8F13C
:102C20000108F7D221464846F4E0FDE00A21C4F34A
:102C300002534FF0000B0891022B07D001CFC117B0
:102C4000032B09D00AE034E023E024E0FF1D27F045
:102C50000707F7E8020105E000B2C117042B01D114
:102C600040B2C117002907DA4FF0000CD0EB0C007E
:102C70006CEB01012D2302E0230504D52B238DF8F5
:102C80002430012303E0E30701D02023F7E798462F
:102C900050E00A210EE010204FF0000B08900CE0ED
:102CA00010214FF0000B44F004044FF00809089184
:102CB00003E008214FF0000B0891C4F30253022BEC
:102CC00004D001CF0021032B06D006E0FF1D27F022
:102CD0000707F7E8020103E080B2042B00D1C0B27D
:102CE0004FF00008230725D5702A2AD0DDF820C030
:102CF0008CF0100C5CEA0B0C09D150EA010306D0F1
:102D000030238DF824308DF8252002239846DDF8F5
:102D100020C08CF0080C5CEA0B0C0BD150EA0103CC
:102D200001D1630706D530238DF824304FF0010818
:102D3000A9F10109582A09D03EA20B9208AA0A92C9
:102D400011E040238DF824300123DFE73EA2F4E7B1
:102D50005B46089AFDF75AFA0B9B9B5C0A9AA2F114
:102D600001020A92137050EA0102F1D10A98ADEB08
:102D7000000000F1200B600702D524F4803401E04C
:102D80004FF00109D94502DDA9EB0B0000E000205E
:102D900000EB0B0141440890AAEB010AE00306D4C2
:102DA000DDE90F232146504600F06BF80644002071
:102DB00008E009A911F80900DDE90F129047761C17
:102DC00009F1010081464045F3DBE0030CD5DDE964
:102DD0000F232146504600F054F8064404E0DDE994
:102DE0000F1230209047761C0899481E0890002941
:102DF000F5DC08E00A980A990078491C0A91DDE997
:102E00000F129047761CBBF10001ABF1010BF1DC16
:102E100021465046DDE90F2300F020F806446D1CE2
:102E2000287800287FF41DAE11B03046BDE8F08F41
:102E30000928010030313233343536373839616290
:102E40006364656600000000303132333435363754
:102E50003839414243444546000000002DE9F04125
:102E6000044600251E461746880405D406E0394668
:102E70002020B04705F10105641EF8D52846BDE8BD
:102E8000F0812DE9F041044600251E469046C80316
:102E900001D5302700E02027880405D506E041460B
:102EA0003846B04705F10105641EF8D52846BDE84F
:102EB000F0810A68531C0B6010707047F0B507462C
:102EC0000C461546002606E014F8011B384600F0B3
:102ED00007F80746761CAE42F6D33846F0BD000030
:102EE000024682EA0100C0B2024B33F8100080EAC9
:102EF000222070474833000870B504460D4600BFD5
:102F000040210548FFF72CFB0028F9D00249091D94
:102F10000C80204670BD0000003801403548006834
:102F200035490840B0F1005F5CD100204FF0E0214E
:102F30000861002240F225513048FFF748FB00228B
:102F400040F224412D48FFF742FB002240F2277156
:102F50002A48FFF73CFB002240212848FFF7F7FAF8
:102F6000002240F225512648FFF731FB002240F2B3
:102F700024412348FFF72BFB002240F22771204811
:102F8000FFF725FB002240211D48FFF7E0FA002152
:102F90001C48FDF783FA00211A481430FDF77EFA29
:102FA000002118482830FDF779FA002115483C30F7
:102FB000FDF774FA002113485030FDF76FFA002135
:102FC0001148FEF7B9FC00214FF08040FEF7B4FC39
:102FD00000210E48FEF7B0FCFDF704FD054800F0A7
:102FE0001DF804E00AA0FDF7D3FEFDF7CDFC00BFFD
:102FF000FEE70000004000080000FE2F00380140FE
:103000000048004008000240002C0140000400403D
:103010004E6F20417070320D0A00000010B504465A
:10302000606806490860084600680549086020682D
:10303000FDF791F802480068804710BD500000205D
:1030400054000020FEF772FBFEF7B4F91CE00F48B5
:10305000007848B1FFF786FB00200C49087040F269
:1030600052410B48FDF7A9F80848007920B100202B
:1030700006490871FEF7C8FA0448C07820B100205C
:103080000249C870FEF7D2FCE1E7000030000020E2
:10309000EE04002010B50446240300F0F5F800F01B
:1030A00087F810210B48FDF722FC2020FEF7DCF901
:1030B000C4F30740FEF7D8F9C4F30720FEF7D4F9AC
:1030C000E0B2FEF7D1F910210248FDF712FC00F042
:1030D0006FF810BD000801402DE9F04105460C468F
:1030E000174610211248FDF702FC0B20FEF7BCF931
:1030F000C4F30740FEF7B8F9C4F30720FEF7B4F9AC
:10310000E0B2FEF7B1F9FF20FEF7AEF92870002615
:1031100005E0FF20FEF7A8F9A855701C86B2BE4254
:10312000F7DB10210248FDF7E4FBBDE8F081000069
:10313000000801402DE9F041002400250026002769
:1031400010210F48FDF7D3FB9F20FEF78DF9FF20DC
:10315000FEF78AF90546FF20FEF786F90646FF20AE
:10316000FEF782F9074610210548FDF7C2FB280447
:1031700040EA062040EA07042046BDE8F08100004E
:103180000008014010B5002410210848FDF7AFFBEE
:103190000520FEF769F9FF20FEF766F904461021C5
:1031A0000248FDF7A6FB204610BD000000080140C4
:1031B00010B500BFFFF7E6FF10F0010FFAD110BD08
:1031C0002DE9F74F82B00F46002000900498B0F52B
:1031D000806F02DD05B0BDE8F08F0120284908703E
:1031E0003E0BC7F30B04C4F5805001902046E11755
:1031F00004EB91514FEAA128E11704EB9151891298
:10320000A4EB81211FFA81F9C9F580601FFA80FAC9
:10321000454623E0300300EB85214FF480621948D6
:10322000FFF75AFF4FF0000B0CE009EB0B001549BC
:10323000085CFF2802D001200090D3460BF101006A
:103240001FFA80FBD345F0DB009808B1042503E0AA
:103250004FF4806A4FF00009681C85B2042DD9DB59
:10326000009810B13046FFF715FF04EB0631049AC1
:10327000029800F019F800200149087000BFA9E782
:1032800018000020A400002010B510210548FDF70B
:103290002EFB0620FEF7E8F810210248FDF729FB77
:1032A00010BD0000000801402DE9F04107460E4620
:1032B0001446F0B2C0F58075AC4200DC254612E041
:1032C0002A463146384600F013F8AC4200D10BE0F4
:1032D0002F442E44601B84B2B4F5807F02DD4FF48E
:1032E000807500E02546EBE700BFBDE8F0810000F7
:1032F0002DE9F04106460C461746FFF7C5FF1021A1
:103300001048FDF7F4FA0220FEF7AEF8C4F30740C8
:10331000FEF7AAF8C4F30720FEF7A6F8E0B2FEF71E
:10332000A3F8002504E0705DFEF79EF8681C85B2E6
:10333000BD42F8DB10210348FDF7DBFAFFF738FF49
:10334000BDE8F081000801400000C1C081C140011A
:1033500001C3C003800241C201C6C006800741C745
:103360000005C1C581C4400401CCC00C800D41CD15
:10337000000FC1CF81CE400E000AC1CA81CB400BE5
:1033800001C9C009800841C801D8C018801941D9B5
:10339000001BC1DB81DA401A001EC1DE81DF401F45
:1033A00001DDC01D801C41DC0014C1D481D5401555
:1033B00001D7C017801641D601D2C012801341D365
:1033C0000011C1D181D0401001F0C030803141F1F5
:1033D0000033C1F381F240320036C1F681F7403745
:1033E00001F5C035803441F4003CC1FC81FD403D15
:1033F00001FFC03F803E41FE01FAC03A803B41FBE5
:103400000039C1F981F840380028C1E881E9402934
:1034100001EBC02B802A41EA01EEC02E802F41EF44
:10342000002DC1ED81EC402C01E4C024802541E554
:103430000027C1E781E640260022C1E281E3402364
:1034400001E1C021802041E001A0C060806141A174
:103450000063C1A381A240620066C1A681A7406744
:1034600001A5C065806441A4006CC1AC81AD406D14
:1034700001AFC06F806E41AE01AAC06A806B41ABE4
:103480000069C1A981A840680078C1B881B94079B4
:1034900001BBC07B807A41BA01BEC07E807F41BF44
:1034A000007DC1BD81BC407C01B4C074807541B554
:1034B0000077C1B781B640760072C1B281B3407364
:1034C00001B1C071807041B00050C19081914051F4
:1034D0000193C053805241920196C0568057419744
:1034E0000055C19581944054019CC05C805D419D14
:1034F000005FC19F819E405E005AC19A819B405BE4
:103500000199C059805841980188C0488049418933
:10351000004BC18B818A404A004EC18E818F404F43
:10352000018DC04D804C418C0044C1848185404553
:103530000187C047804641860182C0428043418363
:103540000041C181818040408000000000000000F7
:10355000000000000000000000000000000000006B
:10356000000000000000000000000000000000005B
:10357000000000000000000000000000000000004B
:103580000000000000000000A83500080000002036
:10359000A4000000342A00084C360008A4000020D3
:1035A0004C130000442A0008000000000000000046
:1035B000000000000000000000000000000000000B
:1035C00000000000000000000000000000000000FB
:1035D00000000000000000000000000000000000EB
:1035E00000000000000000000000000000000000DB
:1035F00000000000000000000000000000000000CB
:1036000000000000000000000000000000000000BA
:1036100000000000000000000000000000000000AA
:103620000000000000000000010203040102030486
:10363000060708090204060800366E0100000000B3
:0C36400000000000010203040607080956
:0400000508000131BD
:00000001FF
